:10245D000001FF00FF000001010000FF00FF01006F
:08246D00102030405060708027
:1020DC004102720041027D0041027B004102780006
:1020EC004102B000C103C189C107C18BC108C10441
:1020FC00C10A4402740000000043020B000024419A
:07210C000202004102A720BE
:1012C50074C12DF58274023CF583E0FFE925E0FB4E
:1012D500EF4BF9224F25E0FFE04F25E0FF224F2598
:1012E500E0FFE04F25E0FF22EFF090020B120E32F7
:1012F500900273E0F582758300020C992BF8E6FFE6
:10130500E0FEEF8EF0A4FFAEF0E4FCFD224F25E0F9
:10131500FFE04F25E0FF22E0FF2424F8E6FE744AB3
:101325002FF582E43402F583224F25E0FFE04F25B7
:10133500E0FF224F25E0FFE04F25E0FF22E025E01A
:1013450024B1F582E43402F5832290020B120E32A9
:10135500900273E0229003DAE0FFA3E0FDA3E0FB37
:10136500229002A7E0FF9003D9E06F2290030BE0E3
:101375002405FFE433FE90030AE0C39FEE6480F882
:10138500748098224F25E0FFE04F25E0FF22120DE3
:10139500A8020D6B90027BE0FF2403F582E4340282
:1013A500F5832274FFF090030AE004F0229002B066
:1013B500E0243CF582E43402F58322900278E024AF
:1013C50044F582E43402F58322900272E0240EF59E
:1013D50082E43402F58322F090027BE075F005A4E7
:1013E50022900273E0FF2424F82290030CE0FFC34F
:1013F5009428227E0012244590030CE004F0222458
:101405005DF582EE3424F583E493FF900397F02293
:1014150090020B020E32747E2DF582740222900327
:101425000BE0FFC3942822120DE990030AE0FB228A
:1014350090027CE0244CF822F582E43402F5832204
:07144500E4334F25E0FF2214
:101CE300E4900273F0D209D20BD206D201D205D20C
:101CF300001213B2E4F01213C0E4F01213CEE4F0B6
:101D030090027BE012139EE4F07F2890027E740120
:101D1300F0A3DFFC7F0490020F7401F0A3DFFC7FCC
:101D2300079002047401F0A3DFFC7F289002C174C2
:101D330001F0A3DFFC7F049002457401F0A3DFFCF4
:0B1D43007F0790023D7401F0A3DFFC5D
:011D4E002272
:031A240002144C5D
:10144C00C0E0C0F0C083C082C0D075D000C000C066
:10145C0001C002C003C004C005C006C007C2DF2023
:05146C00DA0330DB5B38
:10147100900396E5A0F0C2DBC2DA900309E0FF9089
:101481000396E0FE6F540C6042EE13135403FDEF1C
:10149100540CFF7E00ED4F1214049002A6E0FE9062
:1014A1000398F09002A62FF0E06E30E116900397BA
:1014B100E07F04B4010512224D800312248BD20A6D
:0B14C10012251A900396E0900309F03A
:0614CC0020D80330D967AF
:1014D200900396E5A0F0C2D9C2D8900249E0FF90ED
:1014E2000396E0FD6F5403604EEF75F004A47E0096
:1014F200540CFFED5403FDEF4D12140490023BE037
:10150200FE900398F090023B2FF0E06E30E12090C5
:101512000397E07F04B40105121D4F8003121E6A77
:10152200900273E0FFE4FD121636D20A12251A90D9
:071532000396E0900249F06E
:10153900D007D006D005D004D003D002D001D00006
:0B154900D0D0D082D083D0F0D0E032B0
:1023DF0075DA3175DB3175DC3175DD31E49002A6CC
:0A23EF00F043F61075D982D2DE2209
:1025070075BC4075E8C075BA1F75D108E4F5BB43C3
:03251700E60822B1
:0A25990075A14075F80175A2072234
:091A0F00E4F5B1F5A975B28322DA
:0D256A0075921E7593FF75910443E6802263
:0D254E00E4FF74242FF876FF0FEFB428F59A
:01255B00225D
:10214E0078317C037D017BFF7A24796D7E007F08D8
:10215E00120C5AE4FFEF75F005842431F582E43455
:10216E0003F583E0FE74132FF582E43402F583EE5B
:06217E00F00FEFB428DFB2
:012184002238
:1023C30075A4CDE4F5F275F3FF75D4C875D5FF7523
:0C23D300F41F75A70175E10675E24422B5
:0D255C00E4FF744C2FF8E4F60FEFB428F5FF
:01256900224F
:0A2583007F109002B1E4F0A3DFFC2A
:01258D00222B
:10236300E4F5D9121A0F1223C3121CE31225071224
:10237300256A1223DF12259912214E122583022189
:01238300BA9F
:10248B00121435E6FED394045004E4F68004C3EE34
:05249B009FF6022185FF
:10224D0090027CE0FE244CF8E6FDEF2DFDE433FC1E
:10225D00C3ED94FFEC648094804008744C2EF876A6
:0C226D00FF8006121435EF26F6022185D2
:101D4F009003991212EDB4FF0C1213E676E31213FF
:101D5F002374E3804B1212EFD39403500B1213E64C
:101D6F00E4F6121323E4803812134FFF29F9E43AF3
:101D7F00FA120C80FE900399E0FDC3EE9D120CF950
:101D8F001214158F821212FBFF900273E0FE2424AF
:101D9F00F8A6078E821212FBFF744A2E121326EF3B
:051DAF00F012221E22CB
:101E6A009003991212EDC394E3400C1213E676FF25
:101E7A0012132374FF803C1212EF700C1213E676D1
:101E8A00031213237403802B900399E0FF12134F5C
:101E9A00FEF582758300EF120CC68E821212FBFFCA
:101EAA0074242EF8A6078E821212FBFF744A2E1291
:081EBA001326EFF012221E2294
:10252D00121435E6700476FF8002E4F6122185025E
:02253D00251A5D
:101F6C0012134FFF1212F990020BB4FF0C120E3227
:101F7C008F827583007423800A121352F582758345
:101F8C000074FF120D0B12134FFF1212F9FE742482
:101F9C002FF8A606900273E0FF1212F9121322EE2C
:101FAC00F012221E900273E0FFE4FD121636022599
:011FBC001A0A
:05163600900399EFF0A4
:10163B00E490039EF0C216C21753E6EFEDB4010817
:10164B00D2169003997427F0EDB40206D217C2B0EC
:10165B008002D2B0900399E0FD75F00584E5F004AB
:10166B0090039CF0ED75F0058404A3F0D287C2863D
:10167B0090039B7408F0C2831225A320176A900372
:10168B009A7405F090039AE0FFC39401405A9003BB
:10169B009DE0FE90039BE0FDB50607A3E0FEEF6E19
:1016AB0060033016311214159003991212F8C454BA
:1016BB000FFFEDC454F04FFF1225AB12141590031E
:1016CB00991212F8C454F0FF1225AB301612900386
:1016DB0099E014F0800AE4FF1225ABE4FF1225AB6E
:1016EB0090039AE014F0809CA2179218121FBD125F
:1016FB0025A3D28390039BE014F0E0C39401400335
:0B170B000216811225A3C2B043E610B5
:0117160022B0
:0725A300E4FF0FEFB464FB3D
:0125AA00220E
:0825AB00E5A120E7FB8FA3224C
:101FBD00201805E4FF1225AB900202E04430FF1219
:101FCD0025AB121342E0C4F854F0C8A3E0C4540F7B
:101FDD0048FF1225AB900202121342A3E0C4F8543D
:101FED000FC868FF0582D58202158315821225ABB5
:0B1FFD00900202E004F0B40502E4F0E2
:0120080022B5
:0725CB007D02E4FF02163659
:100E81007E0153E6EFC2B0C287D286C2831225A388
:100E9100EE7003021128120E5B0EC8010EFA020F4A
:100EA10025030F58040F73050F8E060FBE070FE6BB
:100EB10008101A0910470A107D0B10A70C10D10D4C
:100EC10010FA0E00000E9190029FE025E0FF9002C3
:100ED100A4E090029E1212D99002A3E04FF9E4FC23
:100EE100FD74442DF58274021212CC0DBD00010C6B
:100EF100ED64044C70EB0210A190029DE025E0FF2F
:100F01009002A2E090029C1212D99002A1E09002FC
:100F1100D01212E39002CBE09002C612131290029B
:100F2100C1021016900297E025E0FF900292E09036
:100F3100028D121312900288E09002E412132E9097
:100F410002DFE09002DA12132E9002D5E04FF9FF92
:100F51001225AB0E020E91E4FCFD743C2DF582745A
:100F6100021212CC0DBD00010CED64084C70EB02B5
:100F710010A1E4FCFD74032DF58274021212CC0D54
:100F8100BD00010CED64084C70EB0210A1E4FCFD06
:100F9100740E2DF58274021212CC0DBD00010CED00
:100FA10064054C70EB7C007D0212141B1212CC0DF7
:100FB100BD00010CED64054C70EF0210A190027FA1
:100FC100E025E0FF90027EE0900286121338A3E054
:100FD100900285121389900284E0900283121338E3
:100FE10090028C8030900291E0F97C007D0B12140C
:100FF1001B1212CC0DBD00010CED640E4C70EFE91B
:1010010025E0FF900290E090028F1212E3A20912F4
:10101100144590028EE00210767C007D1512141B9F
:101021001212CC0DBD00010CED64194C70EF7C0067
:101031007D1D12141B1212CCED1D70011CED6419E3
:101041004C70EF0210A1A206E43325E0FFA201E4F7
:10105100339002A01213899002A5E04F25E0FF9082
:101061000248E04F25E0FFA20B121445A20512141D
:1010710045A200E4334FF90EFF0211227C007D01ED
:101081001212C50DBD00010CED64054C70F27C001F
:101091007D061212C50DBD00010CED640A4C70F203
:1010A1000EAF010211227C007D0B1212C50DBD0095
:1010B100010CED640F4C70F27C007D131212C5ED32
:1010C1001D70011CED640F4C70F20EAF0102112274
:1010D1007C007D151212C50DBD00010CED64194C8B
:1010E10070F27C007D1D1212C5ED1D70011CED64B6
:1010F100194C70F20EAF0180287C007D1F1212C5C1
:101101000DBD00010CED64234C70F27C007D2712B3
:1011110012C5ED1D70011CED64234C70F2E4FEAFAD
:0F112100011225AB020E91D28343E6100225A3E3
:0B19900090039AEEF0A3EFF030074C3C
:10199B0090039AA3E0FF1225B390039CEF1213DC84
:1019AB002F90039DF090039AA3E0FF12258EEF7505
:1019BB00F007A4FF90039CF012141590039D1212D4
:1019CB00F8D39F40047F0180027F0090039AA3E02D
:0B19DB00247EF582E43402F583EFF077
:1019E6002212141590039AE0FEA3E0FFF5828E837F
:1019F600120C99B4FF047D0180027D00747E2FF5E0
:091A060082E43402F583EDF022C4
:10244500AD07744C2DF8E670047C0180027C0074A5
:08245500C12D12143DECF02230
:10221E0012134FFF1212F9FEB4FF06D201D206803E
:10222E0019EE7006D201C2068010EED3942340063A
:0F223E00C201D2068004C201C2067E00021990BE
:1021850090027CE0FF244CF8E6FE700DD200D205EB
:1021950074C12F12143D7401F0EED39400400FC2A8
:1021A50000D20590027CE024C112143DE4F0EEB4A7
:0421B500FF02C2055E
:0121B9002203
:0A258E00EF75F0058475F005A4FF59
:012598002220
:0825B300EF75F00584AFF02282
:101E1100C209E4FD7C2890024A74FFF0A3DCFCEFC8
:101E21003395E0FE7C007D05120D2DAC06AD07EF6C
:101E31002405FBE43EFAC3ED9BEA6480F8EC648080
:101E410098501974242DF8E6FB744A2DF58274021A
:101E51003CF583EBF00DBD00010C80D37B017A02D0
:081E6100794A90020B120E52A7
:011E69002256
:0F253F00D2097B007A00792490020B120E5222EF
:1006A700122363122413E49003CEF0122475D2AF01
:1006B70043E601E490030CF01213EF500A7E001298
:1006C70019901213FD80F1E490030CF01213EF5010
:1006D700051213F880F612221E122185C207C208DE
:1006E700D20AC2B0120B6553E6EFE5147003020895
:1006F7000B24FE700302077D24FA70030207A92466
:10070700F870030207CA240C60030207F112139959
:100717007401F090027DEFF090027BE004F0E0D3EB
:1007270094074002E4F0121399E4F0EF75F005A482
:10073700FF900272E02FFFA3F07E0012199030079E
:100747005CE490030AF090030AE0FFC39428500882
:100757001213231213A880EE1213DD90030BF090EF
:10076700030AF0121371500912131CEE1213AA8018
:10077700F2120B6580271213CE7401F0900272E01B
:1007870004F0E0D394044002E4F0900272E0FF1218
:1007970013D2E41213DCFEEF2E900273F012221E26
:1007A700804820030CE49003CEF0121A1BD20B8072
:1007B70039A208B39208300806C21CC20B802BD29C
:1007C7000B8027A207B3920730070A90027BE0FF4E
:1007D700121E11800312253FE490030BF01214231D
:1007E7005005120B6D80F6120B82300712E490034E
:1007F7000BF01214235005120B6D80F6120B82E4D6
:10080700F514D20AE513607B24E0601224E0603E11
:1008170024C0600F24707066121F6C0208851225B1
:100827002D805B1213B27401F09002B0E004F0E087
:10083700D394074002E4F09002B0E0FF1213B6E44D
:10084700F0EF75F005A4FF900278E02F80291213CE
:10085700C07401F0900278E004F0E0D39404400201
:10086700E4F0900278E0FF1213C4E4F09002B0E0E5
:1008770075F005A4FEEF2E90027CF0122185D20AB6
:10088700E4F513300717E490030BF0121423500D0F
:100897007E0012199090030BE004F080EE20020313
:1008A7000209DBC20243E610E490030AF090030D4D
:1008B700120DF50000000090030AE0FB244CF8E657
:1008C700FF9002A8121305900311120DE9745190BD
:1008D70002A912130190031512142C2456F8E6FFEF
:1008E7009002AA121305900319120DE9745B900286
:1008F700AB12130190031D12142C2460F8E6FF902D
:1009070002AC121305900321120DE974652BF8E66A
:10091700FF9002AD12130590032512142C246AF8D8
:10092700E6FF9002AE121305900329120DE9746FCA
:100937002BF8E6FF9002AF12130590032D120DE975
:10094700900315120D9C9003111213939003191223
:10095700139390031D121393900321121393900383
:100967002512139390032912139390032D121393B7
:1009770090030D120DE9E47FFF7EFFFDFC90030D50
:10098700120DA8D3120D78400A90030D120DF50031
:1009970000FFFF90030D120D9C7804120D89900340
:1009A7000AE0FD121343EEF0A3EFF0ED121343E05C
:1009B700FEA3E0C394FFEE940F400BED12134374B4
:1009C7000FF0A374FFF01213ABE064056003020895
:1009D700B41225CB1221EEEF7003020B579003D808
:1009E700E0FFB40B05D203020AC0EF64317029128D
:1009F70013666003020AC012233F50FB120B7912E1
:100A0700233F50FB12135AA3E0900334F01217F759
:100A170012233F50FB020A9A9003D8E06432701DFC
:100A27001213666003020AC012233F50FB120B79B0
:100A370012135A1218C612233F50FB80569003D840
:100A4700E0642D7024121366706F12233F50FB90E1
:100A570002A7E0FF1224CA12233F50FB12135A12B7
:100A67001ACE12233F50FB802A9003D8E0642E70E1
:100A77002C121366704312233F50FB9002A7E0FF2E
:100A87001224CA12233F50FB12135A121A30122390
:100A97003F50FB9002A7E0FF1224B5801C9003D8BB
:100AA700E0FFB4140AD208C20BC21CD20A800AEFB4
:100AB700B41506C208D20BD20A200803020B5790BE
:100AC70003D8E0146075046003020B579003D9E064
:100AD7009003CEF0122475E490030AF090030AE025
:100AE700FFC3942850081213231213A880EE121381
:100AF700DD90030BF090030AF012137150091213E3
:100B07001CEE1213AA80F2E490030CF01213EF50BC
:100B17000A7E001219901213FD80F1E490030CF085
:100B27001213EF50051213F880F612221E122185B8
:100B3700D20A7D01E4FF12163680159003D9E090A2
:030B470003CEF0EA
:0D0B4A00A2AF920DC2AF121A1BA20D92AF06
:0E0B5700200A030206EE120E81C20A0206EE0A
:100B65007D01E4FF121636227E0012199090030BC8
:100B7500E004F0229002A7E0FF1224CA227D01E4DE
:050B8500FF12163622EC
:101B6500E5B0541EF512650E600CE512650EF5160E
:101B750075113285120EE51160431511E511703DA1
:101B8500E51630E108E51220E103751402E516308B
:101B9500E208E51220E203751404E51630E311E5C9
:101BA5001220E30C900279740BF0A374B8F0D20CF8
:101BB500E51630E408E51220E403751410300C2D09
:101BC50090027974FFF5F0120D3FE5B030E305752D
:101BD5001408C20C900279E07002A3E0700FC20CE9
:0E1BE50030030A9002A7E0FF7D131223842232
:101EC200E5A054F0F510650D600CE510650DF515F3
:101ED200750F3285100DE50F603A150FE50F70345E
:101EE200E51530E408E51020E403751310E515301C
:101EF200E508E51020E503751320E51530E608E551
:101F02001020E603751340E51530E708E51020E7D9
:051F120003751380229D
:031A2D0002205440
:10205400C0E0C0F0C083C082C0D075D000C000C052
:1020640001C002C003C004C005C006C00753917F6D
:10207400121B65121EC275BB0075E8D0D007D006CE
:10208400D005D004D003D002D001D000D0D0D0826B
:07209400D083D0F0D0E03250
:031A210002200997
:10200900C0E0C083C082C0D075D000C006C007C27E
:10201900EDE5BB64086025E5BEC4333354C0FFE574
:10202900BD1313543F4FFFAEBB74A82EF582E434A1
:1020390002F583EFF005BB75E8D08002D202D00724
:0B204900D006D0D0D082D083D0E0328F
:10171700902B0075F050ED120E26EC75F050A425B5
:1017270083AF8290033DF0A3EFF0900335E075F0AF
:1017370050A42400F9742B35F0FA7BFF22E075F0F2
:1017470050902B00120E26AF82AE8322900389E4BD
:1017570075F001020D3F900332E475F001120E3B64
:10176700AE02AF01227B007A007924900339E4F0BE
:10177700A322E024FFFFE434FFFE900336E0FCA33E
:10178700E0FD22900389E0FCA3E0FDC39450EC94B4
:101797000022E475F001120D5585F082F583E4937C
:1017A7002224FFFEE434FF900336F0A3CEF022900C
:1017B700033A120E52E4900338F0A3F022AD04ED81
:1017C700FFEEF0A3EFF022E4900389F0A3F022AF3D
:1017D70005E4F0A3EFF0E07F00FE2274372DF582D9
:1017E700E43403F583229FEE6480F8EC648098224A
:101C6C009003317403F0E4A3F0A3F01225BB7E348F
:101C7C007F607B017A03793112177204F0122116FE
:101C8C007B007A007924900338120DF50000005087
:101C9C00E4FD12231B12254E12255CE4900332F056
:101CAC00900332E0FFC3941E501875F050EF1217DA
:101CBC004812176C7450F0122116900332E004F0A5
:101CCC0080DE7E347F617B017A03793312177204D4
:071CDC00F01221160222F5AF
:10251A00201C0F3003083008071225C38002C20BA3
:03252A00D21C229E
:10241300903461E493600C903460E493640360034C
:09242300121C6CE49003CEF022BF
:102475009003CE12173478247C007D007E007F50B7
:06248500120C5AC21C22D9
:1024A0001225BB9003CE12174412176C7450F01211
:0524B00021160222F5D7
:061A1B001224A0C21C22EF
:0817F700900331EFF0A3EDF0C7
:1017FF00A2AFE43390033FF0C2AF900331E0FFD3C9
:10180F009B4033EF1217A8EB14900335F09003327F
:10181F00121779D31217ED50581217171217B61255
:10182F00188B40FB1222F590033612175690033592
:10183F00E004F002181C900332E01217A890033452
:10184F00E014A3F0900331121779C31217ED402162
:10185F001217171217B612188B40FB1222F59003AE
:10186F003674FFF5F0120D3F900335E014F00218B7
:0C187F005390033FE024FF92AF0221BA17
:10188B0090033AE475F001120E3BAE02AF019003E8
:10189B003DE475F001120D5585F082F583E493FD5F
:1018AB00121BF3900338E475F001120D3FC3900344
:0B18BB0039E09450900338E0940022C4
:0518C600900331EDF07C
:1018CB00A2AFE43390038BF0C2AFEF14900387F019
:1018DB00EB14A3F0900331E014FF900387E0D39F48
:1018EB004003021985A31217441217CE12178A5000
:1018FB00190FEFAA0670010E14F5828A83E493FB8D
:10190B001217E2EBF012175380E290038812173490
:10191B00900332120E52900387121744900335EE48
:10192B00F0A3EFF01217CE12175D90033512179933
:10193B00FD121BF3121753C390038AE094509003CC
:10194B0089E0940040E19003871217349003321220
:10195B000E521217CE12178A501012175D1217E281
:10196B00E0FD121BF312175380EB1222F590038745
:10197B00E004F0A3E004F00218DF90038BE024FFF7
:05198B0092AF0221BA39
:071A3000900331EBF0AC075D
:101A3700A2AFE43390033BF0C2AF9003321217D644
:101A4700900332F0A3EFF09003321217C490033AD9
:101A5700740FF01225BB90033A1217349003361215
:101A67000E52E4900334F0A3F0900332E0FCA3E0BD
:101A7700FFECFD900331E0FBE490033FF0D20E1240
:101A87001554900339EFF0FD900336121760121BBF
:101A9700F3900332121756900334121756C390036C
:101AA70035E09450900334E0940040BD1222F59045
:101AB700033AE004F0E0C3941E40981221BA900361
:061AC7003BE024FF92AF9A
:011ACD0022F6
:071ACE00900331EBF0AC07BF
:101AD500A2AFE433900339F0C2AF9003341217D6A6
:101AE500900334F0A3EFF09003341217C490033839
:101AF500740FF0900338E0FFC3941E505775F050F3
:101B0500EF121748900336EEF0A3EFF0E49003329E
:101B1500F0A3F0900334E0FCA3E0FFECFD9003316B
:101B2500E0FB90033612179990033FF0C20E121591
:101B350054900334121756900332121756C390036C
:101B450033E09450900332E0940040C7900338E0AE
:0F1B550004F0809F1221BA900339E024FF92AF71
:011B6400225E
:05231B00900337EDF016
:1023200090033874FF120DB6EC4D4E4F60109003C1
:0E23300037E0120CF9740129F9E43AFA80E260
:01233E00227C
:1023A400E475F001120D5585F082F5832275B7A509
:0F23B40075B7F18F828E8322EEF0A3EFF0A32294
:10242C00A2AFE433FDC2AF758F031223B1E4F0F514
:08243C008FAF05EF24FF92AF02
:012444002275
:1023F900A2AFE433FCC2AF758F011223B1EDF0E453
:09240900F58FAF04EF24FF92AF40
:0124120022A7
:10209B009003921223BCECF0A3EDF0EB4A6031906D
:1020AB000392E0FEA3E0FFA3E0FCA3E0F5828C83A8
:1020BB00E0FD1223F9EB1B70011A900394E475F009
:1020CB0001120D3F900392E475F001120D3F80CB8E
:0120DB0022E2
:0825BB00E4900000F0A3F022FF
:1022F500900000E0FEA3E0FF12242C900000E0FE19
:10230500A3E0FF7C007D027B007A0212209BE49013
:062315000000F0A3F0221D
:0A1BF300A90590038CEEF0A3EFF0BB
:101BFD00EE54FEFE900000E0FCA3E0FD7002EE6CE2
:101C0D006044ED4C60031222F590038CE0FEEE541F
:101C1D00FEFE7F00900000F0A3EFF090038E1223E4
:101C2D00BC7400F0A37402F07F007E0290038E124C
:101C3D0023A4E493FD9003901223A4EDF0EF1F7005
:101C4D00011EEF4E70E690038CE0FCA3E0FDEC541A
:0E1C5D0001FC74022DF58274003CF583E9F061
:011C6B002256
:102116009003341223BC120E5290033974FFF5F06B
:10212600120D5545F06020900334E475F001120D50
:1021360055AFF0FE900336E475F001120E3B120C1B
:0821460080FD121BF380D22280
:03000000020600F5
:03000300021A03DB
:03000B00021A06D0
:03001300021A09C5
:03001B00021A0CBA
:03002300021A0FAF
:03002B00021A12A4
:03003300021A1599
:03003B00021A188E
:03004300021A1B83
:03004B00021A1E78
:03005300021A216D
:03005B00021A2462
:03006300021A2757
:03006B00021A2A4C
:03007300021A2D41
:10060000E4F5D9E5EF7480F5FF7402F5EF787FE447
:10061000F6D8FD9000007F007E04E4F0A3DFFCDE4E
:07062000FA75817302066206
:02211300C11AEF
:101F17009003ACE475F001120D5585F082F583222C
:101F27009003A7E0FFA3E0CF9003A3F0A3EFF02275
:101F37009003AC7403F0A374BEF0229003A3E4757E
:101F4700F001120D3F7E037FCE9003A3E022E0FE57
:101F5700A3E0FF9003A3E0FCA3E0FD22EE9003A71C
:051F6700F0A3EFF022E1
:10233F009003A7121F55B50719ECB506159003ACFE
:10234F00E0FEA3E0FFEDB50709ECB5060520C502D9
:04235F00D322C322A0
:0C257700758920438E08758DE8D28E22F5
:1024DF0075C101E4F5C2F5C053C17F43C18043F616
:0424EF00010225774A
:1021BA007E037FAE9003A5EEF0A3EFF09003AAEEA4
:1021CA00F0A3EFF09003A1EEF0A3EFF07E037FBE41
:1021DA00121F639003ACEEF0A3EFF0EE121F2FC2B2
:0421EA00190224DFD3
:1022CE009003AA121F1AEFF09003AA121F1AEDF034
:1022DE009003AAE0B4030FA3E0B4BE0A9003AA745D
:0722EE0003F0A374AEF0221F
:0725D200C219C2C4D2C522E8
:101DB40020192FD219121F1774FFF07C037DCE90C7
:101DC40003ACE0B50408A3E0B50503121F37121FE6
:101DD40017E4F09003ACE0B50408A3E0B5050312E2
:101DE4001F37121F17E4F09003ACE0B40308A3E01C
:101DF400B4CE03121F37121F17EFF09003ACE0B4F8
:0D1E04000308A3E0B4CE03121F377F0122B4
:102279009003A5E0FCA3E0FD9003A1E0B50408A349
:10228900E0B505037F00229003A5E0FCA3E0F582F9
:0C2299008C83E0B507037F01227F002248
:1022A5009003A5E475F001120D3F9003A5121F1AC6
:1022B500E0FF9003A5E0B4030FA3E0B4BE0A9003CA
:0822C500A57403F0A374AEF050
:0122CD0022EE
:061A27007FFF122279226C
:0625D900E4FF122279224A
:031A180002113088
:10113000C0E0C0F0C083C082C0D075D000C000C085
:1011400004C005C006C007E5C054FE120E5B128F36
:1011500008128F0A12A50C12A50E1268101268123E
:10116000128414128416125B1C125B1E1257241276
:101170005726121A28121A2A12282C12282E11BCAD
:10118000C011C6C2118EE0118EE2000012AEC2C5BF
:10119000121F42B5060BA3E0B507069003A3121F6A
:1011A0003A9003A3121F1AE0F5C29003A3E06E70F9
:1011B00003A3E06F60030212AE021211121F27D2C6
:1011C000C4D2C50212AE9003AC121F55B5070EEC87
:1011D000B5060A121F63C2C5D2C40212AE8D828C3C
:1011E00083E0B4FF030212AA121F42B5060BA3E06C
:1011F000B507069003A3121F3A9003A3121F1AE02B
:10120000F5C29003A3E06E7003A3E06F60030212C7
:10121000AE9003A3121F3A0212AEE5C260289002FC
:10122000A7E065C260208013121F27C2C5D21AE54D
:10123000C260139002A7E065C2600BC2C4C2C5C2FF
:10124000C1C21B0212AEADC27FFF1222CEC2C4C207
:10125000C5D2C1D21B8057D2C580539003A3E0FFF3
:10126000A3E0CF121F6480469003AAE0FFA3E090A2
:1012700003A1CFF0A3EFF0C2C4C2C1301A30D2C56F
:10128000C21A802A121F27C2C4C2C1D2C5801FC27F
:10129000C4C2C5201B04C2C18014ADC2E4FF122227
:1012A000CED2C18009121F27C2C1C2C4D2C5C2C0DA
:1012B000D007D006D005D004D000D0D0D082D083C3
:0512C000D0F0D0E03287
:1023840090039FEFF0A3EDF07F0A121DB490039F1A
:10239400E0FF121DB49003A0E0FF121DB40225D289
:0825C3007F02121DB40225D2B3
:0621EE00121A27EF602722
:1021F4009003317403F0A374D7F01222A590033135
:10220400E475F001120D5585F082F583EFF0122587
:07221400D9EF70E67F012203
:03221B007F00221F
:1024B500900331EFF07F2F121DB4900331E0FF122E
:0524C5001DB40225D248
:1024CA00900331EFF07F30121DB4900331E0FF1218
:0524DA001DB40225D233
:1024F300EFFD900341E0FB3395E0FAC3EB9D74805D
:04250300F86A9822B8
:0815540090033CEFF0A3EDF061
:10155C00A20E9212C214201EFDD21E900340EBF07C
:10156C00C20FD210D2137F01C2C4C215D2C530C073
:10157C00FDE5C054F02480607624C0601B24E0603C
:10158C000302161B900340E0F5C2A20FE43342C2E3
:10159C00C2C5E4A3F002161D30C149301507D2C5EF
:1015AC00C21502161D30100CC210D21190033DE072
:1015BC00F5C2805D301111C21190033CE0F5C230D0
:1015CC00124FD215D20F8049200F461224F3500E21
:1015DC0090033FE0F5C2900341E004F08033D2C4A5
:1015EC00C21E802D301304D2C58026D21480221244
:1015FC0024F3500CA3E5C2F0900341E004F0D2C1F7
:10160C00900341E0B5070AC21EC2C1D2C48002D207
:10161C001430140853C0BF43C040C21EC2C0301E99
:09162C000302157A900342E0FF6D
:011635002292
:100627000206A7E493A3F8E493A34003F68001F23C
:1006370008DFF48029E493A3F85407240CC8C333D4
:10064700C4540F4420C8834004F456800146F6DFA3
:10065700E4800B01020408102040809020DCE47E37
:10066700019360BCA3FF543F30E509541FFEE49398
:10067700A360010ECF54C025E060A840B8E493A35F
:10068700FAE493A3F8E493A3C8C582C8CAC583CA8A
:10069700F0A3C8C582C8CAC583CADFE9DEE780BE42
:0121150000C9
:100B8A00E709F608DFFA8046E709F208DFFA803E4D
:100B9A0088828C83E709F0A3DFFA8032E309F6083A
:100BAA00DFFA8078E309F208DFFA807088828C83A2
:100BBA00E309F0A3DFFA806489828A83E0A3F60856
:100BCA00DFFA805889828A83E0A3F208DFFA804C30
:100BDA0080D280FA80C680D4806980F28033801007
:100BEA0080A680EA809A80A880DA80E280CA803370
:100BFA0089828A83ECFAE493A3C8C582C8CCC583E8
:100C0A00CCF0A3C8C582C8CCC583CCDFE9DEE780B7
:100C1A000D89828A83E493A3F608DFF9ECFAA9F036
:100C2A00EDFB2289828A83ECFAE0A3C8C582C8CC8C
:100C3A00C583CCF0A3C8C582C8CCC583CCDFEADEA5
:100C4A00E880DB89828A83E493A3F208DFF980CC07
:100C5A0088F0EF60010E4E60C388F0ED2402B40400
:100C6A000050B9F582EB2402B4040050AF232345A7
:060C7A008223900BDA73E7
:100C8000BB010689828A83E0225002E722BBFE0272
:090C9000E32289828A83E49322A5
:100C9900BB010CE58229F582E5833AF583E0225010
:100CA90006E92582F8E622BBFE06E92582F8E2225A
:0D0CB900E58229F582E5833AF583E4932274
:100CC600BB010FF8E58229F582E5833AF583E02832
:100CD600F0225009C58229F8E58226F622BBFE09D4
:100CE600C58229F8E22582F222F8EA2583F583E90E
:030CF6009328221E
:100CF900BB010689828A83F0225002F722BBFE01DA
:020D0900F322D3
:100D0B00F8BB010DE58229F582E5833AF583E8F01E
:100D1B00225006E92582C8F622BBFE05E92582C8CA
:020D2B00F222B2
:100D2D00EF8DF0A4A8F0CF8CF0A428CE8DF0A42EDA
:020D3D00FE2294
:100D3F00C5F0F8A3E028F0C5F0F8E582158270023F
:060D4F001583E038F022DC
:100D5500A3F8E0C5F025F0F0E58215827002158351
:060D6500E0C838F0E822AE
:0D0D6B00EF2BFFEE3AFEED39FDEC38FC22D7
:100D7800EB9FF5F0EA9E42F0E99D42F0E89C45F0D1
:010D88002248
:100D8900E8600FECC313FCED13FDEE13FEEF13FF48
:030D9900D8F1226C
:0C0D9C00E0FCA3E0FDA3E0FEA3E0FF22CA
:0C0DA800E0F8A3E0F9A3E0FAA3E0FB22CE
:100DB4007401FF3395E0FEFDFCA3A3A3E0CF2FF065
:100DC400E582158270021583E0CE3EF0E58215823D
:100DD40070021583E0CD3DF0E58215827002158323
:050DE400E0CC3CF02210
:0C0DE900ECF0A3EDF0A3EEF0A3EFF0227D
:100DF500A8828583F0D083D082120E0C120E0C12BD
:100E05000E0C120E0CE473E493A3C583C5F0C583E1
:100E1500C8C582C8F0A3C583C5F0C583C8C582C847
:010E250022AA
:0C0E2600A42582F582E5F03583F58322D7
:090E3200E0FBA3E0FAA3E0F922C1
:100E3B00F8E0FBA3A3E0F925F0F0E5821582700240
:070E4B001583E0FA38F022E4
:090E5200EBF0A3EAF0A3E9F022A1
:100E5B00D083D082F8E4937012740193700DA3A326
:100E6B0093F8740193F5828883E47374029368603A
:060E7B00EFA3A3A380DF3A
:00000001FF
